 prefs

 Timestamp is b5cb96b9 (reproducible build file hash)

 Preferred load address is 0000000180000000

 Start         Length     Name                   Class
 0001:00000000 000015c0H .text$mn                CODE
 0001:000015c0 00000036H .text$mn$00             CODE
 0001:000015f6 00000092H .text$x                 CODE
 0002:00000000 00000178H .idata$5                DATA
 0002:00000178 00000038H .00cfg                  DATA
 0002:000001b0 00000008H .CRT$XCA                DATA
 0002:000001b8 00000008H .CRT$XCZ                DATA
 0002:000001c0 00000008H .CRT$XIA                DATA
 0002:000001c8 00000008H .CRT$XIZ                DATA
 0002:000001d0 00000008H .CRT$XPA                DATA
 0002:000001d8 00000008H .CRT$XPZ                DATA
 0002:000001e0 00000008H .CRT$XTA                DATA
 0002:000001e8 00000008H .CRT$XTZ                DATA
 0002:000001f0 00000000H .gehcont$y              DATA
 0002:000001f0 00000000H .gfids$y                DATA
 0002:000001f0 00000210H .rdata                  DATA
 0002:00000400 00000000H .rdata$CastGuardVftablesA DATA
 0002:00000400 00000000H .rdata$CastGuardVftablesC DATA
 0002:00000400 0000006cH .rdata$voltmd           DATA
 0002:0000046c 000002b4H .rdata$zzzdbg           DATA
 0002:00000720 00000008H .rtc$IAA                DATA
 0002:00000728 00000008H .rtc$IZZ                DATA
 0002:00000730 00000008H .rtc$TAA                DATA
 0002:00000738 00000008H .rtc$TZZ                DATA
 0002:00000740 00000220H .xdata                  DATA
 0002:00000960 0000033cH .edata                  DATA
 0002:00000c9c 00000078H .idata$2                DATA
 0002:00000d14 00000014H .idata$3                DATA
 0002:00000d28 00000178H .idata$4                DATA
 0002:00000ea0 000003baH .idata$6                DATA
 0003:00000000 00000040H .data                   DATA
 0003:00000040 000005f8H .bss                    DATA
 0004:00000000 00000234H .pdata                  DATA
 0005:00000000 00000060H .rsrc$01                DATA
 0005:00000060 00000308H .rsrc$02                DATA

  Address         Publics by Value              Rva+Base               Lib:Object

 0000:00000000       __AbsoluteZero             0000000000000000     <absolute>
 0000:00000000       ___safe_se_handler_count   0000000000000000     <absolute>
 0000:00000000       ___safe_se_handler_table   0000000000000000     <absolute>
 0000:00000000       __arm64x_extra_rfe_table   0000000000000000     <absolute>
 0000:00000000       __arm64x_extra_rfe_table_size 0000000000000000     <absolute>
 0000:00000000       __arm64x_native_entrypoint 0000000000000000     <absolute>
 0000:00000000       __arm64x_redirection_metadata 0000000000000000     <absolute>
 0000:00000000       __arm64x_redirection_metadata_count 0000000000000000     <absolute>
 0000:00000000       __dynamic_value_reloc_table 0000000000000000     <absolute>
 0000:00000000       __enclave_config           0000000000000000     <absolute>
 0000:00000000       __guard_check_icall_a64n_fptr 0000000000000000     <absolute>
 0000:00000000       __guard_eh_cont_count      0000000000000000     <absolute>
 0000:00000000       __guard_eh_cont_table      0000000000000000     <absolute>
 0000:00000000       __guard_fids_count         0000000000000000     <absolute>
 0000:00000000       __guard_fids_table         0000000000000000     <absolute>
 0000:00000000       __guard_iat_count          0000000000000000     <absolute>
 0000:00000000       __guard_iat_table          0000000000000000     <absolute>
 0000:00000000       __guard_longjmp_count      0000000000000000     <absolute>
 0000:00000000       __guard_longjmp_table      0000000000000000     <absolute>
 0000:00000000       __hybrid_auxiliary_delayload_iat 0000000000000000     <absolute>
 0000:00000000       __hybrid_auxiliary_delayload_iat_copy 0000000000000000     <absolute>
 0000:00000000       __hybrid_auxiliary_iat     0000000000000000     <absolute>
 0000:00000000       __hybrid_auxiliary_iat_copy 0000000000000000     <absolute>
 0000:00000000       __hybrid_code_map          0000000000000000     <absolute>
 0000:00000000       __hybrid_code_map_count    0000000000000000     <absolute>
 0000:00000000       __hybrid_image_info_bitfield 0000000000000000     <absolute>
 0000:00000000       __x64_code_ranges_to_entry_points 0000000000000000     <absolute>
 0000:00000000       __x64_code_ranges_to_entry_points_count 0000000000000000     <absolute>
 0000:00000100       __guard_flags              0000000000000100     <absolute>
 0000:00000000       __ImageBase                0000000180000000     <linker-defined>
 0001:00000000       Java_java_util_prefs_WindowsPreferences_WindowsRegCloseKey 0000000180001000 f   WindowsPreferences.obj
 0001:0000000c       Java_java_util_prefs_WindowsPreferences_WindowsRegCreateKeyEx 000000018000100c f   WindowsPreferences.obj
 0001:00000118       Java_java_util_prefs_WindowsPreferences_WindowsRegDeleteKey 0000000180001118 f   WindowsPreferences.obj
 0001:0000018c       Java_java_util_prefs_WindowsPreferences_WindowsRegDeleteValue 000000018000118c f   WindowsPreferences.obj
 0001:00000208       Java_java_util_prefs_WindowsPreferences_WindowsRegEnumKeyEx 0000000180001208 f   WindowsPreferences.obj
 0001:000002e8       Java_java_util_prefs_WindowsPreferences_WindowsRegEnumValue 00000001800012e8 f   WindowsPreferences.obj
 0001:000003c8       Java_java_util_prefs_WindowsPreferences_WindowsRegFlushKey 00000001800013c8 f   WindowsPreferences.obj
 0001:000003d4       Java_java_util_prefs_WindowsPreferences_WindowsRegOpenKey 00000001800013d4 f   WindowsPreferences.obj
 0001:000004a8       Java_java_util_prefs_WindowsPreferences_WindowsRegQueryInfoKey 00000001800014a8 f   WindowsPreferences.obj
 0001:000005a0       Java_java_util_prefs_WindowsPreferences_WindowsRegQueryValueEx 00000001800015a0 f   WindowsPreferences.obj
 0001:000006e8       Java_java_util_prefs_WindowsPreferences_WindowsRegSetValueEx 00000001800016e8 f   WindowsPreferences.obj
 0001:000007e2       JNU_ThrowOutOfMemoryError  00000001800017e2 f   java:java.dll
 0001:000007e8       __GSHandlerCheck           00000001800017e8 f   MSVCRT:gshandler.obj
 0001:00000808       __GSHandlerCheckCommon     0000000180001808 f   MSVCRT:gshandler.obj
 0001:00000880       __security_check_cookie    0000000180001880 f   MSVCRT:amdsecgs.obj
 0001:00000bc0       _DllMainCRTStartup         0000000180001bc0 f   MSVCRT:dll_dllmain.obj
 0001:00000c00       __raise_securityfailure    0000000180001c00 f   MSVCRT:gs_report.obj
 0001:00000c34       __report_gsfailure         0000000180001c34 f   MSVCRT:gs_report.obj
 0001:00000d7c       __security_init_cookie     0000000180001d7c f   MSVCRT:gs_support.obj
 0001:00000e28       DllMain                    0000000180001e28 f   MSVCRT:dll_dllmain_stub.obj
 0001:00000e4c       ?__scrt_initialize_type_info@@YAXXZ 0000000180001e4c f   MSVCRT:tncleanup.obj
 0001:00000e5c       ?__scrt_uninitialize_type_info@@YAXXZ 0000000180001e5c f   MSVCRT:tncleanup.obj
 0001:00000e68       __local_stdio_printf_options 0000000180001e68 f i MSVCRT:default_local_stdio_options.obj
 0001:00000e70       __local_stdio_scanf_options 0000000180001e70 f i MSVCRT:default_local_stdio_options.obj
 0001:00000e78       __scrt_initialize_default_local_stdio_options 0000000180001e78 f   MSVCRT:default_local_stdio_options.obj
 0001:00000e94       __scrt_acquire_startup_lock 0000000180001e94 f   MSVCRT:utility.obj
 0001:00000ed0       __scrt_dllmain_after_initialize_c 0000000180001ed0 f   MSVCRT:utility.obj
 0001:00000f04       __scrt_dllmain_before_initialize_c 0000000180001f04 f   MSVCRT:utility.obj
 0001:00000f1c       __scrt_dllmain_crt_thread_attach 0000000180001f1c f   MSVCRT:utility.obj
 0001:00000f44       __scrt_dllmain_crt_thread_detach 0000000180001f44 f   MSVCRT:utility.obj
 0001:00000f5c       __scrt_dllmain_exception_filter 0000000180001f5c f   MSVCRT:utility.obj
 0001:00000fbc       __scrt_dllmain_uninitialize_c 0000000180001fbc f   MSVCRT:utility.obj
 0001:00000fec       __scrt_dllmain_uninitialize_critical 0000000180001fec f   MSVCRT:utility.obj
 0001:00001000       __scrt_initialize_crt      0000000180002000 f   MSVCRT:utility.obj
 0001:0000104c       __scrt_initialize_onexit_tables 000000018000204c f   MSVCRT:utility.obj
 0001:000010d8       __scrt_is_nonwritable_in_current_image 00000001800020d8 f   MSVCRT:utility.obj
 0001:00001170       __scrt_release_startup_lock 0000000180002170 f   MSVCRT:utility.obj
 0001:00001194       __scrt_uninitialize_crt    0000000180002194 f   MSVCRT:utility.obj
 0001:000011c0       __scrt_get_dyn_tls_init_callback 00000001800021c0 f   MSVCRT:dyn_tls_init.obj
 0001:000011c8       __crt_debugger_hook        00000001800021c8 f   MSVCRT:utility_desktop.obj
 0001:000011d0       __scrt_fastfail            00000001800021d0 f   MSVCRT:utility_desktop.obj
 0001:0000131c       _RTC_Initialize            000000018000231c f   MSVCRT:initsect.obj
 0001:00001358       _RTC_Terminate             0000000180002358 f   MSVCRT:initsect.obj
 0001:00001394       _guard_check_icall_nop     0000000180002394 f i MSVCRT:guard_support.obj
 0001:00001398       __isa_available_init       0000000180002398 f   MSVCRT:cpu_disp.obj
 0001:00001544       _get_startup_argv_mode     0000000180002544 f   MSVCRT:argv_mode.obj
 0001:0000154c       __scrt_is_ucrt_dll_in_use  000000018000254c f   MSVCRT:ucrt_detection.obj
 0001:00001560       __C_specific_handler       0000000180002560 f   vcruntime:VCRUNTIME140.dll
 0001:00001566       __std_type_info_destroy_list 0000000180002566 f   vcruntime:VCRUNTIME140.dll
 0001:0000156c       memset                     000000018000256c f   vcruntime:VCRUNTIME140.dll
 0001:00001572       _initterm                  0000000180002572 f   ucrt:api-ms-win-crt-runtime-l1-1-0.dll
 0001:00001578       _initterm_e                0000000180002578 f   ucrt:api-ms-win-crt-runtime-l1-1-0.dll
 0001:0000157e       _seh_filter_dll            000000018000257e f   ucrt:api-ms-win-crt-runtime-l1-1-0.dll
 0001:00001584       _configure_narrow_argv     0000000180002584 f   ucrt:api-ms-win-crt-runtime-l1-1-0.dll
 0001:0000158a       _initialize_narrow_environment 000000018000258a f   ucrt:api-ms-win-crt-runtime-l1-1-0.dll
 0001:00001590       _initialize_onexit_table   0000000180002590 f   ucrt:api-ms-win-crt-runtime-l1-1-0.dll
 0001:00001596       _execute_onexit_table      0000000180002596 f   ucrt:api-ms-win-crt-runtime-l1-1-0.dll
 0001:0000159c       _cexit                     000000018000259c f   ucrt:api-ms-win-crt-runtime-l1-1-0.dll
 0001:000015a4       __acrt_initialize          00000001800025a4 f   MSVCRT:ucrt_stubs.obj
 0001:000015a4       __acrt_thread_attach       00000001800025a4 f   MSVCRT:ucrt_stubs.obj
 0001:000015a4       __acrt_thread_detach       00000001800025a4 f   MSVCRT:ucrt_stubs.obj
 0001:000015a4       __acrt_uninitialize        00000001800025a4 f   MSVCRT:ucrt_stubs.obj
 0001:000015a4       __acrt_uninitialize_critical 00000001800025a4 f   MSVCRT:ucrt_stubs.obj
 0001:000015a4       __scrt_stub_for_acrt_initialize 00000001800025a4 f   MSVCRT:ucrt_stubs.obj
 0001:000015a4       __scrt_stub_for_acrt_thread_attach 00000001800025a4 f   MSVCRT:ucrt_stubs.obj
 0001:000015a4       __scrt_stub_for_acrt_thread_detach 00000001800025a4 f   MSVCRT:ucrt_stubs.obj
 0001:000015a4       __scrt_stub_for_acrt_uninitialize 00000001800025a4 f   MSVCRT:ucrt_stubs.obj
 0001:000015a4       __scrt_stub_for_acrt_uninitialize_critical 00000001800025a4 f   MSVCRT:ucrt_stubs.obj
 0001:000015a4       __vcrt_initialize          00000001800025a4 f   MSVCRT:ucrt_stubs.obj
 0001:000015a4       __vcrt_thread_attach       00000001800025a4 f   MSVCRT:ucrt_stubs.obj
 0001:000015a4       __vcrt_thread_detach       00000001800025a4 f   MSVCRT:ucrt_stubs.obj
 0001:000015a4       __vcrt_uninitialize        00000001800025a4 f   MSVCRT:ucrt_stubs.obj
 0001:000015a4       __vcrt_uninitialize_critical 00000001800025a4 f   MSVCRT:ucrt_stubs.obj
 0001:000015a8       __scrt_stub_for_is_c_termination_complete 00000001800025a8 f   MSVCRT:ucrt_stubs.obj
 0001:000015a8       _is_c_termination_complete 00000001800025a8 f   MSVCRT:ucrt_stubs.obj
 0001:000015ab       memcpy                     00000001800025ab f   vcruntime:VCRUNTIME140.dll
 0001:000015d0       _guard_dispatch_icall_nop  00000001800025d0 f   MSVCRT:guard_dispatch.obj
 0001:000015f0       _guard_xfg_dispatch_icall_nop 00000001800025f0 f   MSVCRT:guard_xfg_dispatch.obj
 0002:00000000       __imp_RegCloseKey          0000000180003000     advapi32:ADVAPI32.dll
 0002:00000008       __imp_RegCreateKeyExA      0000000180003008     advapi32:ADVAPI32.dll
 0002:00000010       __imp_RegDeleteKeyA        0000000180003010     advapi32:ADVAPI32.dll
 0002:00000018       __imp_RegDeleteValueA      0000000180003018     advapi32:ADVAPI32.dll
 0002:00000020       __imp_RegEnumKeyExA        0000000180003020     advapi32:ADVAPI32.dll
 0002:00000028       __imp_RegEnumValueA        0000000180003028     advapi32:ADVAPI32.dll
 0002:00000030       __imp_RegFlushKey          0000000180003030     advapi32:ADVAPI32.dll
 0002:00000038       __imp_RegOpenKeyExA        0000000180003038     advapi32:ADVAPI32.dll
 0002:00000040       __imp_RegQueryInfoKeyA     0000000180003040     advapi32:ADVAPI32.dll
 0002:00000048       __imp_RegQueryValueExA     0000000180003048     advapi32:ADVAPI32.dll
 0002:00000050       __imp_RegSetValueExA       0000000180003050     advapi32:ADVAPI32.dll
 0002:00000058       \177ADVAPI32_NULL_THUNK_DATA 0000000180003058     advapi32:ADVAPI32.dll
 0002:00000060       __imp_RtlCaptureContext    0000000180003060     kernel32:KERNEL32.dll
 0002:00000068       __imp_RtlLookupFunctionEntry 0000000180003068     kernel32:KERNEL32.dll
 0002:00000070       __imp_RtlVirtualUnwind     0000000180003070     kernel32:KERNEL32.dll
 0002:00000078       __imp_UnhandledExceptionFilter 0000000180003078     kernel32:KERNEL32.dll
 0002:00000080       __imp_SetUnhandledExceptionFilter 0000000180003080     kernel32:KERNEL32.dll
 0002:00000088       __imp_GetCurrentProcess    0000000180003088     kernel32:KERNEL32.dll
 0002:00000090       __imp_TerminateProcess     0000000180003090     kernel32:KERNEL32.dll
 0002:00000098       __imp_IsProcessorFeaturePresent 0000000180003098     kernel32:KERNEL32.dll
 0002:000000a0       __imp_QueryPerformanceCounter 00000001800030a0     kernel32:KERNEL32.dll
 0002:000000a8       __imp_GetCurrentProcessId  00000001800030a8     kernel32:KERNEL32.dll
 0002:000000b0       __imp_GetCurrentThreadId   00000001800030b0     kernel32:KERNEL32.dll
 0002:000000b8       __imp_GetSystemTimeAsFileTime 00000001800030b8     kernel32:KERNEL32.dll
 0002:000000c0       __imp_DisableThreadLibraryCalls 00000001800030c0     kernel32:KERNEL32.dll
 0002:000000c8       __imp_InitializeSListHead  00000001800030c8     kernel32:KERNEL32.dll
 0002:000000d0       __imp_IsDebuggerPresent    00000001800030d0     kernel32:KERNEL32.dll
 0002:000000d8       \177KERNEL32_NULL_THUNK_DATA 00000001800030d8     kernel32:KERNEL32.dll
 0002:000000e0       __imp_memset               00000001800030e0     vcruntime:VCRUNTIME140.dll
 0002:000000e8       __imp_memcpy               00000001800030e8     vcruntime:VCRUNTIME140.dll
 0002:000000f0       __imp___C_specific_handler 00000001800030f0     vcruntime:VCRUNTIME140.dll
 0002:000000f8       __imp___std_type_info_destroy_list 00000001800030f8     vcruntime:VCRUNTIME140.dll
 0002:00000100       \177VCRUNTIME140_NULL_THUNK_DATA 0000000180003100     vcruntime:VCRUNTIME140.dll
 0002:00000108       __imp_free                 0000000180003108     ucrt:api-ms-win-crt-heap-l1-1-0.dll
 0002:00000110       __imp_malloc               0000000180003110     ucrt:api-ms-win-crt-heap-l1-1-0.dll
 0002:00000118       \177api-ms-win-crt-heap-l1-1-0_NULL_THUNK_DATA 0000000180003118     ucrt:api-ms-win-crt-heap-l1-1-0.dll
 0002:00000120       __imp__initterm            0000000180003120     ucrt:api-ms-win-crt-runtime-l1-1-0.dll
 0002:00000128       __imp__initterm_e          0000000180003128     ucrt:api-ms-win-crt-runtime-l1-1-0.dll
 0002:00000130       __imp__seh_filter_dll      0000000180003130     ucrt:api-ms-win-crt-runtime-l1-1-0.dll
 0002:00000138       __imp__configure_narrow_argv 0000000180003138     ucrt:api-ms-win-crt-runtime-l1-1-0.dll
 0002:00000140       __imp__initialize_narrow_environment 0000000180003140     ucrt:api-ms-win-crt-runtime-l1-1-0.dll
 0002:00000148       __imp__initialize_onexit_table 0000000180003148     ucrt:api-ms-win-crt-runtime-l1-1-0.dll
 0002:00000150       __imp__execute_onexit_table 0000000180003150     ucrt:api-ms-win-crt-runtime-l1-1-0.dll
 0002:00000158       __imp__cexit               0000000180003158     ucrt:api-ms-win-crt-runtime-l1-1-0.dll
 0002:00000160       \177api-ms-win-crt-runtime-l1-1-0_NULL_THUNK_DATA 0000000180003160     ucrt:api-ms-win-crt-runtime-l1-1-0.dll
 0002:00000168       __imp_JNU_ThrowOutOfMemoryError 0000000180003168     java:java.dll
 0002:00000170       \177java_NULL_THUNK_DATA   0000000180003170     java:java.dll
 0002:00000178       __guard_check_icall_fptr   0000000180003178     MSVCRT:guard_support.obj
 0002:00000180       __guard_xfg_check_icall_fptr 0000000180003180     MSVCRT:guard_support.obj
 0002:00000188       __guard_dispatch_icall_fptr 0000000180003188     MSVCRT:guard_support.obj
 0002:00000190       __guard_xfg_dispatch_icall_fptr 0000000180003190     MSVCRT:guard_support.obj
 0002:00000198       __guard_xfg_table_dispatch_icall_fptr 0000000180003198     MSVCRT:guard_support.obj
 0002:000001a0       __castguard_check_failure_os_handled_fptr 00000001800031a0     MSVCRT:guard_support.obj
 0002:000001a8       __guard_memcpy_fptr        00000001800031a8     vcruntime:softmemtag.obj
 0002:000001b0       __xc_a                     00000001800031b0     MSVCRT:initializers.obj
 0002:000001b8       __xc_z                     00000001800031b8     MSVCRT:initializers.obj
 0002:000001c0       __xi_a                     00000001800031c0     MSVCRT:initializers.obj
 0002:000001c8       __xi_z                     00000001800031c8     MSVCRT:initializers.obj
 0002:000001d0       __xp_a                     00000001800031d0     MSVCRT:initializers.obj
 0002:000001d8       __xp_z                     00000001800031d8     MSVCRT:initializers.obj
 0002:000001e0       __xt_a                     00000001800031e0     MSVCRT:initializers.obj
 0002:000001e8       __xt_z                     00000001800031e8     MSVCRT:initializers.obj
 0002:000001f0       ??_C@_0CA@NIIGFDJD@native?5memory?5allocation?5failed@ 00000001800031f0     WindowsPreferences.obj
 0002:00000210       _pDefaultRawDllMain        0000000180003210     MSVCRT:dll_dllmain.obj
 0002:00000210       _pRawDllMain               0000000180003210     MSVCRT:dll_dllmain.obj
 0002:00000230       __xmm@ffffffffffffffffffffffffffffffff 0000000180003230     MSVCRT:utility.obj
 0002:00000240       _load_config_used          0000000180003240     MSVCRT:loadcfg.obj
 0002:00000400       __volatile_metadata        0000000180003400     <linker-defined>
 0002:00000720       __rtc_iaa                  0000000180003720     MSVCRT:initsect.obj
 0002:00000728       __rtc_izz                  0000000180003728     MSVCRT:initsect.obj
 0002:00000730       __rtc_taa                  0000000180003730     MSVCRT:initsect.obj
 0002:00000738       __rtc_tzz                  0000000180003738     MSVCRT:initsect.obj
 0002:00000c9c       __IMPORT_DESCRIPTOR_ADVAPI32 0000000180003c9c     advapi32:ADVAPI32.dll
 0002:00000cb0       __IMPORT_DESCRIPTOR_java   0000000180003cb0     java:java.dll
 0002:00000cc4       __IMPORT_DESCRIPTOR_KERNEL32 0000000180003cc4     kernel32:KERNEL32.dll
 0002:00000cd8       __IMPORT_DESCRIPTOR_VCRUNTIME140 0000000180003cd8     vcruntime:VCRUNTIME140.dll
 0002:00000cec       __IMPORT_DESCRIPTOR_api-ms-win-crt-heap-l1-1-0 0000000180003cec     ucrt:api-ms-win-crt-heap-l1-1-0.dll
 0002:00000d00       __IMPORT_DESCRIPTOR_api-ms-win-crt-runtime-l1-1-0 0000000180003d00     ucrt:api-ms-win-crt-runtime-l1-1-0.dll
 0002:00000d14       __NULL_IMPORT_DESCRIPTOR   0000000180003d14     advapi32:ADVAPI32.dll
 0003:00000000       __security_cookie_complement 0000000180005000     MSVCRT:gs_cookie.obj
 0003:00000008       __security_cookie          0000000180005008     MSVCRT:gs_cookie.obj
 0003:00000010       __scrt_native_dllmain_reason 0000000180005010     MSVCRT:utility.obj
 0003:00000018       __isa_available            0000000180005018     MSVCRT:cpu_disp.obj
 0003:0000001c       __isa_enabled              000000018000501c     MSVCRT:cpu_disp.obj
 0003:00000020       __memset_fast_string_threshold 0000000180005020     MSVCRT:cpu_disp.obj
 0003:00000028       __memset_nt_threshold      0000000180005028     MSVCRT:cpu_disp.obj
 0003:00000030       __scrt_ucrt_dll_is_in_use  0000000180005030     MSVCRT:ucrt_stubs.obj
 0003:000005c0       ?__type_info_root_node@@3U__type_info_node@@A 00000001800055c0     MSVCRT:tncleanup.obj
 0003:000005d0       ?_OptionsStorage@?1??__local_stdio_printf_options@@9@4_KA 00000001800055d0     MSVCRT:default_local_stdio_options.obj
 0003:000005d8       ?_OptionsStorage@?1??__local_stdio_scanf_options@@9@4_KA 00000001800055d8     MSVCRT:default_local_stdio_options.obj
 0003:000005e0       __scrt_current_native_startup_state 00000001800055e0     MSVCRT:utility.obj
 0003:000005e8       __scrt_native_startup_lock 00000001800055e8     MSVCRT:utility.obj
 0003:00000628       __scrt_debugger_hook_flag  0000000180005628     MSVCRT:utility_desktop.obj
 0003:0000062c       __favor                    000000018000562c     MSVCRT:cpu_disp.obj
 0003:00000630       __dyn_tls_init_callback    0000000180005630     <common>

 entry point at        0001:00000bc0

 Static symbols

 0000:ffff7000       .debug$S                   0000000180000000     prefs.exp
 0000:ffff7000       .debug$S                   0000000180000000     vcruntime:VCRUNTIME140.dll
 0000:ffff7000       .debug$S                   0000000180000000     vcruntime:VCRUNTIME140.dll
 0000:ffff7000       .debug$S                   0000000180000000     vcruntime:VCRUNTIME140.dll
 0000:ffff7000       .debug$S                   0000000180000000     vcruntime:VCRUNTIME140.dll
 0000:ffff7000       .debug$S                   0000000180000000     vcruntime:VCRUNTIME140.dll
 0000:ffff7000       .debug$S                   0000000180000000     vcruntime:VCRUNTIME140.dll
 0000:ffff7000       .debug$S                   0000000180000000     ucrt:api-ms-win-crt-heap-l1-1-0.dll
 0000:ffff7000       .debug$S                   0000000180000000     ucrt:api-ms-win-crt-heap-l1-1-0.dll
 0000:ffff7000       .debug$S                   0000000180000000     ucrt:api-ms-win-crt-runtime-l1-1-0.dll
 0000:ffff7000       .debug$S                   0000000180000000     ucrt:api-ms-win-crt-runtime-l1-1-0.dll
 0000:ffff7000       .debug$S                   0000000180000000     ucrt:api-ms-win-crt-runtime-l1-1-0.dll
 0000:ffff7000       .debug$S                   0000000180000000     ucrt:api-ms-win-crt-runtime-l1-1-0.dll
 0000:ffff7000       .debug$S                   0000000180000000     ucrt:api-ms-win-crt-runtime-l1-1-0.dll
 0000:ffff7000       .debug$S                   0000000180000000     ucrt:api-ms-win-crt-runtime-l1-1-0.dll
 0000:ffff7000       .debug$S                   0000000180000000     ucrt:api-ms-win-crt-runtime-l1-1-0.dll
 0000:ffff7000       .debug$S                   0000000180000000     ucrt:api-ms-win-crt-runtime-l1-1-0.dll
 0000:ffff7000       .debug$S                   0000000180000000     ucrt:api-ms-win-crt-runtime-l1-1-0.dll
 0000:ffff7000       .debug$S                   0000000180000000     ucrt:api-ms-win-crt-runtime-l1-1-0.dll
 0000:ffff7000       .debug$S                   0000000180000000     ucrt:api-ms-win-crt-runtime-l1-1-0.dll
 0000:ffff7000       .debug$S                   0000000180000000     ucrt:api-ms-win-crt-runtime-l1-1-0.dll
 0000:ffff7000       .debug$S                   0000000180000000     advapi32:ADVAPI32.dll
 0000:ffff7000       .debug$S                   0000000180000000     advapi32:ADVAPI32.dll
 0000:ffff7000       .debug$S                   0000000180000000     advapi32:ADVAPI32.dll
 0000:ffff7000       .debug$S                   0000000180000000     advapi32:ADVAPI32.dll
 0000:ffff7000       .debug$S                   0000000180000000     advapi32:ADVAPI32.dll
 0000:ffff7000       .debug$S                   0000000180000000     advapi32:ADVAPI32.dll
 0000:ffff7000       .debug$S                   0000000180000000     advapi32:ADVAPI32.dll
 0000:ffff7000       .debug$S                   0000000180000000     advapi32:ADVAPI32.dll
 0000:ffff7000       .debug$S                   0000000180000000     advapi32:ADVAPI32.dll
 0000:ffff7000       .debug$S                   0000000180000000     advapi32:ADVAPI32.dll
 0000:ffff7000       .debug$S                   0000000180000000     advapi32:ADVAPI32.dll
 0000:ffff7000       .debug$S                   0000000180000000     kernel32:KERNEL32.dll
 0000:ffff7000       .debug$S                   0000000180000000     kernel32:KERNEL32.dll
 0000:ffff7000       .debug$S                   0000000180000000     kernel32:KERNEL32.dll
 0000:ffff7000       .debug$S                   0000000180000000     kernel32:KERNEL32.dll
 0000:ffff7000       .debug$S                   0000000180000000     kernel32:KERNEL32.dll
 0000:ffff7000       .debug$S                   0000000180000000     kernel32:KERNEL32.dll
 0000:ffff7000       .debug$S                   0000000180000000     kernel32:KERNEL32.dll
 0000:ffff7000       .debug$S                   0000000180000000     kernel32:KERNEL32.dll
 0000:ffff7000       .debug$S                   0000000180000000     kernel32:KERNEL32.dll
 0000:ffff7000       .debug$S                   0000000180000000     kernel32:KERNEL32.dll
 0000:ffff7000       .debug$S                   0000000180000000     kernel32:KERNEL32.dll
 0000:ffff7000       .debug$S                   0000000180000000     kernel32:KERNEL32.dll
 0000:ffff7000       .debug$S                   0000000180000000     kernel32:KERNEL32.dll
 0000:ffff7000       .debug$S                   0000000180000000     kernel32:KERNEL32.dll
 0000:ffff7000       .debug$S                   0000000180000000     kernel32:KERNEL32.dll
 0000:ffff7000       .debug$S                   0000000180000000     kernel32:KERNEL32.dll
 0000:ffff7000       .debug$S                   0000000180000000     kernel32:KERNEL32.dll
 0000:ffff7000       .debug$S                   0000000180000000     java:java.dll
 0001:00000870       $$000000                   0000000180001870     MSVCRT:amdsecgs.obj
 0001:000008a0       ?dllmain_crt_dispatch@@YAHQEAUHINSTANCE__@@KQEAX@Z 00000001800018a0 f   MSVCRT:dll_dllmain.obj
 0001:000008f0       ?dllmain_crt_process_attach@@YAHQEAUHINSTANCE__@@QEAX@Z 00000001800018f0 f   MSVCRT:dll_dllmain.obj
 0001:00000a08       ?dllmain_crt_process_detach@@YAH_N@Z 0000000180001a08 f   MSVCRT:dll_dllmain.obj
 0001:00000a8c       ?dllmain_dispatch@@YAHQEAUHINSTANCE__@@KQEAX@Z 0000000180001a8c f   MSVCRT:dll_dllmain.obj
 0001:00000d08       capture_previous_context   0000000180001d08 f   MSVCRT:gs_report.obj
 0001:000015c0       $$000000                   00000001800025c0     MSVCRT:guard_dispatch.obj
 0001:000015e0       $$000000                   00000001800025e0     MSVCRT:guard_xfg_dispatch.obj
 0001:000015f6       ?fin$0@?0??dllmain_crt_process_attach@@YAHQEAUHINSTANCE__@@QEAX@Z@4HA 00000001800025f6 f   MSVCRT:dll_dllmain.obj
 0001:0000160d       ?fin$0@?0??dllmain_crt_process_detach@@YAH_N@Z@4HA 000000018000260d f   MSVCRT:dll_dllmain.obj
 0001:00001626       ?fin$1@?0??dllmain_crt_process_detach@@YAH_N@Z@4HA 0000000180002626 f   MSVCRT:dll_dllmain.obj
 0001:0000163a       ?filt$0@?0??dllmain_dispatch@@YAHQEAUHINSTANCE__@@KQEAX@Z@4HA 000000018000263a f   MSVCRT:dll_dllmain.obj
 0001:00001670       __scrt_is_nonwritable_in_current_image$filt$0 0000000180002670 f   MSVCRT:utility.obj
 0002:00000218       GS_ExceptionPointers       0000000180003218     MSVCRT:gs_report.obj
 0002:00000740       $unwind$Java_java_util_prefs_WindowsPreferences_WindowsRegOpenKey 0000000180003740     WindowsPreferences.obj
 0002:00000754       $unwind$Java_java_util_prefs_WindowsPreferences_WindowsRegCreateKeyEx 0000000180003754     WindowsPreferences.obj
 0002:0000076c       $unwind$Java_java_util_prefs_WindowsPreferences_WindowsRegDeleteKey 000000018000376c     WindowsPreferences.obj
 0002:0000076c       $unwind$Java_java_util_prefs_WindowsPreferences_WindowsRegDeleteValue 000000018000376c     WindowsPreferences.obj
 0002:0000076c       $unwind$__scrt_dllmain_exception_filter 000000018000376c     MSVCRT:utility.obj
 0002:00000780       $unwind$Java_java_util_prefs_WindowsPreferences_WindowsRegQueryValueEx 0000000180003780     WindowsPreferences.obj
 0002:00000794       $unwind$Java_java_util_prefs_WindowsPreferences_WindowsRegSetValueEx 0000000180003794     WindowsPreferences.obj
 0002:000007b0       $unwind$Java_java_util_prefs_WindowsPreferences_WindowsRegQueryInfoKey 00000001800037b0     WindowsPreferences.obj
 0002:000007cc       $unwind$Java_java_util_prefs_WindowsPreferences_WindowsRegEnumKeyEx 00000001800037cc     WindowsPreferences.obj
 0002:000007cc       $unwind$Java_java_util_prefs_WindowsPreferences_WindowsRegEnumValue 00000001800037cc     WindowsPreferences.obj
 0002:000007e4       $unwind$__GSHandlerCheckCommon 00000001800037e4     MSVCRT:gshandler.obj
 0002:000007ec       $unwind$__scrt_initialize_default_local_stdio_options 00000001800037ec     MSVCRT:default_local_stdio_options.obj
 0002:000007ec       $unwind$?dllmain_crt_dispatch@@YAHQEAUHINSTANCE__@@KQEAX@Z 00000001800037ec     MSVCRT:dll_dllmain.obj
 0002:000007ec       $unwind$DllMain            00000001800037ec     MSVCRT:dll_dllmain_stub.obj
 0002:000007ec       $unwind$__GSHandlerCheck   00000001800037ec     MSVCRT:gshandler.obj
 0002:000007ec       $unwind$__scrt_acquire_startup_lock 00000001800037ec     MSVCRT:utility.obj
 0002:000007ec       $unwind$__scrt_dllmain_after_initialize_c 00000001800037ec     MSVCRT:utility.obj
 0002:000007ec       $unwind$__scrt_dllmain_before_initialize_c 00000001800037ec     MSVCRT:utility.obj
 0002:000007ec       $unwind$__scrt_dllmain_crt_thread_attach 00000001800037ec     MSVCRT:utility.obj
 0002:000007ec       $unwind$__scrt_dllmain_crt_thread_detach 00000001800037ec     MSVCRT:utility.obj
 0002:000007ec       $unwind$__scrt_dllmain_uninitialize_c 00000001800037ec     MSVCRT:utility.obj
 0002:000007ec       $unwind$__scrt_dllmain_uninitialize_critical 00000001800037ec     MSVCRT:utility.obj
 0002:000007f8       $xdatasym                  00000001800037f8     MSVCRT:amdsecgs.obj
 0002:000007fc       $unwind$?dllmain_crt_process_attach@@YAHQEAUHINSTANCE__@@QEAX@Z 00000001800037fc     MSVCRT:dll_dllmain.obj
 0002:00000838       $unwind$?fin$0@?0??dllmain_crt_process_attach@@YAHQEAUHINSTANCE__@@QEAX@Z@4HA 0000000180003838     MSVCRT:dll_dllmain.obj
 0002:00000838       $unwind$?fin$0@?0??dllmain_crt_process_detach@@YAH_N@Z@4HA 0000000180003838     MSVCRT:dll_dllmain.obj
 0002:00000838       $unwind$?fin$1@?0??dllmain_crt_process_detach@@YAH_N@Z@4HA 0000000180003838     MSVCRT:dll_dllmain.obj
 0002:00000840       $unwind$?dllmain_crt_process_detach@@YAH_N@Z 0000000180003840     MSVCRT:dll_dllmain.obj
 0002:00000894       $unwind$?dllmain_dispatch@@YAHQEAUHINSTANCE__@@KQEAX@Z 0000000180003894     MSVCRT:dll_dllmain.obj
 0002:000008bc       $unwind$?filt$0@?0??dllmain_dispatch@@YAHQEAUHINSTANCE__@@KQEAX@Z@4HA 00000001800038bc     MSVCRT:dll_dllmain.obj
 0002:000008c4       $unwind$_DllMainCRTStartup 00000001800038c4     MSVCRT:dll_dllmain.obj
 0002:000008d4       $unwind$__report_gsfailure 00000001800038d4     MSVCRT:gs_report.obj
 0002:000008dc       $unwind$capture_previous_context 00000001800038dc     MSVCRT:gs_report.obj
 0002:000008e8       $unwind$__raise_securityfailure 00000001800038e8     MSVCRT:gs_report.obj
 0002:000008e8       $unwind$__scrt_initialize_crt 00000001800038e8     MSVCRT:utility.obj
 0002:000008e8       $unwind$__scrt_initialize_onexit_tables 00000001800038e8     MSVCRT:utility.obj
 0002:000008e8       $unwind$__scrt_release_startup_lock 00000001800038e8     MSVCRT:utility.obj
 0002:000008e8       $unwind$__scrt_uninitialize_crt 00000001800038e8     MSVCRT:utility.obj
 0002:000008f0       $unwind$__security_init_cookie 00000001800038f0     MSVCRT:gs_support.obj
 0002:000008fc       $unwind$__scrt_is_nonwritable_in_current_image 00000001800038fc     MSVCRT:utility.obj
 0002:0000091c       $unwind$__scrt_is_nonwritable_in_current_image$filt$0 000000018000391c     MSVCRT:utility.obj
 0002:00000924       $unwind$__scrt_fastfail    0000000180003924     MSVCRT:utility_desktop.obj
 0002:00000934       $unwind$_RTC_Initialize    0000000180003934     MSVCRT:initsect.obj
 0002:00000934       $unwind$_RTC_Terminate     0000000180003934     MSVCRT:initsect.obj
 0002:00000940       $unwind$__isa_available_init 0000000180003940     MSVCRT:cpu_disp.obj
 0002:00000950       $xdatasym                  0000000180003950     MSVCRT:guard_dispatch.obj
 0002:00000958       $xdatasym                  0000000180003958     MSVCRT:guard_xfg_dispatch.obj
 0002:00000960       .edata                     0000000180003960     prefs.exp
 0002:00000988       rgpv                       0000000180003988     prefs.exp
 0002:000009b4       rgszName                   00000001800039b4     prefs.exp
 0002:000009e0       rgwOrd                     00000001800039e0     prefs.exp
 0002:000009f6       szName                     00000001800039f6     prefs.exp
 0002:00000a00       $N00001                    0000000180003a00     prefs.exp
 0002:00000a3b       $N00002                    0000000180003a3b     prefs.exp
 0002:00000a79       $N00003                    0000000180003a79     prefs.exp
 0002:00000ab5       $N00004                    0000000180003ab5     prefs.exp
 0002:00000af3       $N00005                    0000000180003af3     prefs.exp
 0002:00000b2f       $N00006                    0000000180003b2f     prefs.exp
 0002:00000b6b       $N00007                    0000000180003b6b     prefs.exp
 0002:00000ba6       $N00008                    0000000180003ba6     prefs.exp
 0002:00000be0       $N00009                    0000000180003be0     prefs.exp
 0002:00000c1f       $N00010                    0000000180003c1f     prefs.exp
 0002:00000c5e       $N00011                    0000000180003c5e     prefs.exp
 0002:00000f5a       .idata$6                   0000000180003f5a     advapi32:ADVAPI32.dll
 0002:00000f84       .idata$6                   0000000180003f84     java:java.dll
 0002:000010f4       .idata$6                   00000001800040f4     kernel32:KERNEL32.dll
 0002:00001144       .idata$6                   0000000180004144     vcruntime:VCRUNTIME140.dll
 0002:0000120e       .idata$6                   000000018000420e     ucrt:api-ms-win-crt-heap-l1-1-0.dll
 0002:0000122e       .idata$6                   000000018000422e     ucrt:api-ms-win-crt-runtime-l1-1-0.dll
 0003:00000040       ?__proc_attached@@3HA      0000000180005040     MSVCRT:dll_dllmain.obj
 0003:00000050       GS_ExceptionRecord         0000000180005050     MSVCRT:gs_report.obj
 0003:000000f0       GS_ContextRecord           00000001800050f0     MSVCRT:gs_report.obj
 0003:000005f0       ?is_initialized_as_dll@@3_NA 00000001800055f0     MSVCRT:utility.obj
 0003:000005f1       ?module_local_atexit_table_initialized@@3_NA 00000001800055f1     MSVCRT:utility.obj
 0003:000005f8       ?module_local_atexit_table@@3U_onexit_table_t@@A 00000001800055f8     MSVCRT:utility.obj
 0003:00000610       ?module_local_at_quick_exit_table@@3U_onexit_table_t@@A 0000000180005610     MSVCRT:utility.obj
 0005:00000060       $R000000                   0000000180007060     prefs.dll.res
